:1000000000308A0001290000831A0A28A500030E87
:10001000A6000F288312A500030EA600A6140A0846
:10002000AD008A018313A50E0408A7002008A800CC
:100030002108A9002208AA002308AB002408AC006C
:1000400083128B1E25280B193A28270884002808BC
:10005000A0002908A1002A08A2002B08A3002C0850
:10006000A4002D088A00260E83008312250EA618F0
:1000700083160900AE08031D4028AF08031949285C
:100080002E0F45282F0F452849282E080319AF03A6
:10009000AE03AE08031D5728AF08031D57280030D4
:1000A000051A0130003A03195728B00159280130C8
:1000B000B0000B118A1125283A0883169B009C1367
:1000C0001C141A088312BB0001303A07BC008316C7
:1000D0009B009C131C141A088312BD003B08A3004C
:1000E0003D08A1003B08A2000034113083168F00A8
:1000F00017308312980064001F1300308038831675
:1001000091001F169F161F1383129F171F1407308D
:10011000990083160508831219088C11831699011A
:100120003F30850095008113093087000108C039F0
:100130000738810083128B16C0308B04B801851CF0
:10014000B80A0310B80D0030051D0130B8040310C3
:10015000380DB900BA005C202208B2002108B100B5
:10016000B801051CB80A0310B80D0030851E013017
:10017000B8040310380D083EB900BA005C2022080C
:10018000B4002108B3000712871207111429383070
:10019000840000080319D2280930A000A00BCE2843
:1001A000800BCC280034380DA000A00DFC30A00539
:1001B0001F08C33920049F00BA01B901BB013B08E5
:1001C000073C031CF4289F149F18E42883161E087C
:1001D0008312B9071E0803181E0FBA07D030A000FB
:1001E000A00BF028BB0ADF28BA0CB90CBA0CB90C6A
:1001F000BA0CB90C1F30BA053908A1003A08A200A0
:10020000322984011F308305113083168F00831239
:1002100087141F1300308316910007308312990052
:10022000AF01AE01B0017528B5013508093C031CCA
:10023000242964008716C830B800C7208712C83048
:10024000B800C720B50A152964000B138B138B1B4C
:1002500026292F08B7002E08B600C0308B040730BF
:10026000B800D3282208B9002108B80032083902A2
:10027000031C4B29031D40293808310203184B2960
:1002800007150B138B138B1B4229FF30AF00AE00F9
:10029000C0308B045A290711360F5A29370F5A29B3
:1002A0000B138B138B1B51293408AF003308AE009E
:1002B000C0308B046400B008031D61290712871247
:1002C00070290716B608031D6829B70803196F2996
:1002D000360F6D29370F6D296F2987167029871200
:0402E000242963006A
:104200000200F2000300050003002C00030042003E
:10421000000001000000900001001F0002003D00AE
:08422000000000000000010095
:02400E00CC33B1
:00000001FF
